:10026B00E4F516F514F5171203371201B8D2E8901E
:10027B00E668E04409F090E65C742CF090E65E745E
:10028B0050F0D2AF000000E4FFFEE4FDFC7580806F
:10029B00E4F5800DBD00010CE4B505F1ECB408EDFF
:1002AB00E4FCFDE4F5800DBD00010CE4B505F4ECB8
:1002BB00B408F00FBF00010EEF64014E70CCE514D3
:1002CB00700875B10A75808280F4E5166401702799
:1002DB00F51675B10A90E680E0F50A5488FFBF80E9
:1002EB000B75B1D5E4F51585158080D275B1D57533
:1002FB00150285158080C7E4FFFE90E680E0F50AC5
:10030B000FBF00010EEF64644E70EF85158080AE59
:1003370090E6007412F0A37443F075808275B28260
:0703470075B10A75B6FF2233
:1000920000000090E6047480F00000007402F0009A
:1000A20000007404F00000007406F0000000740800
:0700B200F0000000E4F02261
:1001B80000000000000000000090E6047480F000D9
:1001C80000000000007404F00000007406F0000055
:1001D800007408F0000000E4F000000000000000D7
:1001E800000090E61274A0F000000090E618741168
:1001F800F000000090E61474E0F000000090E61AA9
:10020800740DF000000090E680E0FF5488FEBE8088
:100218000B90E6247402F0E4A3F08009E490E6244D
:10022800F0A37440F000000090E6137422F0000080
:100238000090E6157460F000000090E6097403F081
:10024800BE800B90E6347490F0E4A3F0800A90E648
:10025800347480F0A37440F090E6027460F0A374E4
:0302680008F02279
:10034E00C0E0C083C0825391EF90E65D7401F0D09F
:06035E0082D083D0E032E2
:10031B00C0E0C083C0825391EF90E65D7404F0752A
:0C032B001401751601D082D083D0E0329E
:10036400C0E0C083C0825391EF90E65D7402F0D088
:0603740082D083D0E032CC
:10037A00C0E0C083C0825391EF90E65D7410F0D064
:06038A0082D083D0E032B6
:1000DB00C0E0C083C0825391EF90E65D7408F07569
:0F00EB001601751400751700D082D083D0E03253
:1000B900C0E0C083C0825391EF90E65DE030E50572
:1000C9007420F080F4751601751701D082D083D0A1
:0200D900E03213
:01003F00328E
:01004000328D
:01004100328C
:01004200328B
:01005200327B
:0100FA0032D3
:10000300C0E0C083C082C0D075D000C006C00775F1
:100013008080E4FFFE90E680E0F5080FBF00010E4C
:10002300EF640A4E70EF5391EF90E65F7410F0D0D7
:0C00330007D006D0D0D082D083D0E032BD
:0100FB0032D2
:10005600C0E0C083C082C0D075D000C006C007759E
:100066008080E4FFFE90E680E0F5080FBF00010EF9
:10007600EF640A4E70EF5391EF90E65F7440F0D054
:0C00860007D006D0D0D082D083D0E0326A
:0100FC0032D1
:0100FD0032D0
:0100FE0032CF
:0100FF0032CE
:01039000323A
:010391003239
:010392003238
:010393003237
:010394003236
:010395003235
:010396003234
:010397003233
:010398003232
:010399003231
:01039A003230
:01039B00322F
:01039C00322E
:01039D00322D
:01039E00322C
:01039F00322B
:0103A000322A
:0103A1003229
:0103A2003228
:0103A3003227
:0103A4003226
:0103A5003225
:0103A6003224
:03004300020100B7
:03005300020100A7
:1001000002034E000203640002031B000200DB0036
:1001100002037A000200B90002003F000200400022
:100120000200410002004200020052000200FA00F8
:10013000020003000200FB00020056000200FC0067
:100140000200FD00020040000200FE000200FF006D
:100150000203900002039100020392000203930045
:100160000203940002004000020040000200400030
:100170000203950002039600020397000203980011
:100180000203990002039A0002039B0002039C00F1
:1001900002039D0002039E0002039F000203A000D1
:1001A0000203A1000203A2000203A3000203A400B1
:0801B0000203A5000203A600F2
:03000000020046B5
:0C004600787FE4F6D8FD75811702026B8C
:00000001FF
